:020000040000fa
:0800000082050400000000006d
:020000040000fa
:020000040002f8
:04afe000dfff00008f
:020000040000fa
:020000040002f8
:04afe400ffff00006b
:020000040000fa
:020000040002f8
:04afe80078ff0000ee
:020000040000fa
:020000040002f8
:04afec007dff0000e5
:020000040000fa
:020000040002f8
:04aff00078ff0000e6
:020000040000fa
:1000080000000000000000000000000000000000e8
:100018007a05000000000000000000000000000059
:10002800de09000000000000000000006a0a00006d
:1000380000000000000000000000000000000000b8
:100048009a0a000000000000000000006a0b00008f
:10005800d60b0000060c00000000000000000000a5
:100068000000000000000000000000000000000088
:100078000000000000000000000000000000000078
:10008800000000000000000000000000c60a000098
:100098003a0b000000000000000000000000000013
:1000a8000000000000000000000000000000000048
:1000b8000000000000000000000000000000000038
:1000c8000000000000000000000000000000000028
:1000d8000000000000000000000000000000000018
:1000e8000000000000000000000000000000000008
:1000f80000000000000000000000000000000000f8
:1001080000000000000000000000000000000000e7
:1001180000000000000000000000000000000000d7
:1001280000000000a20b000000000000000000001a
:1001380000000000000000000000000000000000b7
:1001480000000000000000000000000000000000a7
:100158000000000000000000000000000000000097
:100168000000000000000000000000000000000087
:100178000000000000000000000000000000000077
:100188000000000000000000000000000000000067
:1001980000000000000000006e0c00009a0c000037
:1001a800c60c000000000000000000000000000075
:1001b8000000000000000000000000000000000037
:1001c8000000000000000000000000000000000027
:1001d8000000000000000000000000000000000017
:1001e8000000000000000000000000000000000007
:1001f80000000000000000000000000000000000f7
:1002080000000000000000000000000000000000e6
:1002180000000000000000000000000000000000d6
:1002280000000000000000000000000000000000c6
:1002380000000000000000000000000000000000b6
:1002480000000000000000000000000000000000a6
:100258000000000000000000000000000000000096
:100268000000000000000000000000000000000086
:0c0278000000000000000000000000007a
:020000040000fa
:10040000803e2000030007008100e900fcff3a0065
:1004100000000600831f7800c20320000400bc0017
:1004200066015100e0815900f23fb1000380b10044
:1004300006003500ee03090000000000423fb10055
:100440000380b100fbff3d001200b000223fb0006e
:10045000020035000280090000000000cf01780092
:1004600000000600861f78006022b8000602200007
:100470000000d0008180d2000482d2008582d200a8
:100480000000a0000202520083825a0003003100e3
:100490000202420083824a000000a1000603e90034
:1004a000f3ff3a004f03780000000600889fbe006b
:1004b0008a9fbe008c1f78000004be004101070027
:1004c0000478a30026003a006120e10025003200f4
:1004d00009f8a30025003a006420e1002100320061
:1004e000f507b1000508a30002003200000040003b
:1004f000818048006044b800031020000200200002
:1005000000004000818048000805440089854c00b7
:100510000a0541008b8549000a0550008b8558006b
:10052000030033000a00be000204740083847400d8
:100530008301d1000281d300830f7100f0ff3a00e4
:100540008904d1000884d300600149008201780049
:10055000c1adde00fb07b0002f0107000700370028
:100560000960a0000800be0004003700120220004d
:1005700062928800f0ff2f00f1ff27004f067800fd
:100580004f05be004f04be000000060003f0a200ad
:10059000869fbe00889fbe008a9fbe008c9fbe00c3
:1005a00000010700420133006450e1004f003200b7
:1005b0006420e1005200320003826c0007003b001f
:1005c0000905d0000306d000820f54000c065d0020
:1005d0000200390002003200890178000306780029
:1005e0008582550004003d000003fd008103fd00ed
:1005f0008502ea008b854200840f720002003b00f6
:1006000060001000e08018006011b8000005eb00e9
:100610007a28e1000a00390006007800c75ddd0095
:10062000f707b200878075002d00370082817100c6
:100630000a017800610560008180d1000080d3004c
:100640008502e900f9ff3b0006044000878448006a
:1006500002003b0060041400e0841c000988a30031
:10066000070032008a81710082817100610164009b
:100670008904d1000884d3008b05e80017003700f7
:100680000978a30013003a000b00e00013003400c7
:100690008b05e9000804440089844c000a44740076
:1006a0000978a3000d003a000b00e00007003400b9
:1006b0008b05e9000804440089844c0001003a00dd
:1006c0000b0020000978a300f7ff32000001eb00c7
:1006d00002003700828171000a017800ce00070015
:1006e0000cf0a70001f0a000fa0037006420e10040
:1006f00002003a00838f6c00fb0033000801be004b
:100700000200be00f3003700869fbe00889fbe0037
:100710008a9fbe008c9fbe00a2000700e400330049
:1007200003866c006450e100240032006420e10084
:10073000270032006150e100220032006120e10018
:10074000210032008b854200eb07b1000134b80074
:10075000003ab8000804420089844a00013ab8000f
:100760000030b8008880400009014a0004003300ce
:100770000000400081804800020149008b05e9002b
:10078000c909dd0083017000010032001300200060
:10079000c814de004814dd004709de001200b20074
:1007a000c808de00088470009b00070001f0a1006b
:1007b0000cf0a70001f0a000c60037006120e100a6
:1007c000c90032000801be000200be00f7ff37007a
:1007d0006150e100fcff3a00c3003700829fbe0079
:1007e0000001be00770007000470a70003f0a1001d
:1007f0006509b100180032000e0035006828e100dc
:1008000007003500f0ff2f00f1ff27000300e00094
:1008100015003b00010028004f01be00000005004c
:1008200000004000818048008502e900fcff3a009a
:1008300009003700f88f420003003c008000eb0005
:100840004f01be00000005008100d1000080d300f0
:100850008502e800fcff3a000300e00002003b00d4
:1008600060001000e08018004f01be00000006008c
:10087000829fbe000001be00520007000470a70066
:1008800003f0a10003f8a30015003a006509b100c8
:10089000110032000a0035006928e100030035002c
:1008a000010028004f01be000000050000004000cc
:1008b000818048008502e900fcff3a00060037000d
:1008c000f88f4200060035008100d1000080d3007f
:1008d0008502e800fcff3a004f01be000000060060
:1008e0008000eb004f01be00000005008000eb001f
:1008f000829fbe00889fbe008a9fbe0001057800cf
:100900000100e0000400350008003c000000e000a9
:10091000200032000500370060001000e080180061
:1009200002003b0001f024001a0037000004be0062
:100930006011b8006b0920000982cf000200390065
:100940000882cf000441b000694252000e0032001c
:1009500008003b0082817100610164008904d100bc
:100960000884d3008b05e8000442e800f9ff3a0050
:10097000050037000804440089844c008b05e90019
:100980000442e900fbff3a00230007000af0a70039
:1009900001f0a0004f05be004f04be004f01be0095
:1009a000000006000004be00060007000003be00b1
:1009b0000405be000200be0002000700844f75005f
:1009c00000000600c70ade00f107b200f50fb20012
:1009d00008003200e1cf4200020032000170a000a6
:1009e00024000500810f700001003200040805009a
:1009f00044000500810f700002003a001400050059
:100a00008502e9000000400081c04800fcff3b0077
:100a10000170a000240005008100200061805500c5
:100a20000b003d000b00200061fe2f000100e100e3
:100a30001d00340082817100610164008904d100cd
:100a40000884d3000000e800faff3a00710020009b
:100a500061006400030070000200600009003200c1
:100a600061044400e0844c000988a50005003200c0
:100a70008b05e8006808e10002003a008904d10013
:100a80000884d300f20f20000258e10005003d0069
:100a9000c75ddd00f907b2008980750008007800a5
:100aa000000006000bf827008b007800000005000e
:100ab0000200be006450e100050036006420e10041
:100ac000020036000968a30001003a000800be00d9
:100ad0000160a0004f06be004f05be004f04be00df
:100ae0004f03be0000000600f0ff2f00f1ff2700bb
:100af000f8ff37000020ef000220ef00c088a900b7
:100b0000004006000f002100403221000001880053
:100b1000000000000000eb00000778000c00090056
:100b2000002f78000007eb005420ef000e2eef009e
:100b30001e2eef000000eb0001242100bf1d090064
:100b40008018780040a7a900a10020002cfe070013
:100b5000e0022000303a880044e7a90044c7a90019
:100b60004407a9004427a9004447a9004467a900f5
:100b70004487a900300020000600fc0031742000ea
:100b800082072000a309200082487800834878006b
:100b900080487800113a8000618070000600fc00f7
:100ba0002174200062042000730520008248780030
:100bb00083487800804878004427ef00e002200056
:100bc000303a8800300020000d00fc003174200015
:100bd00082072000a309200082487800834878001b
:100be000804878000000200021742000620420006a
:100bf0007305200082487800834878008048780098
:100c000042a7ae00feff3700813e2000fcfd07003a
:100c100010c0b30086e6b70090c2b300c4e6b700c8
:100c2000000ea800007825008070880010cea90072
:100c3000108ea90010aea900008ea9004188a8005e
:100c400041a8a90041c8a90004a1a8000481a800e6
:100c500005e1a8000068a9000021ef0002a1ef0053
:100c60002068a8001061a8001021a90011e1a800c7
:100c700011a1a90010a1a8001081a8000621ef0071
:100c80000a21ef000ca1ef000ea1ef004408a9001b
:100c90004428a9004448a9000108a9002108a80087
:100ca0001fe1a8001fa1a9001ec1a9001ea1a80044
:100cb0001e81a8001e61a9001e21a9004d88a80060
:100cc0004da8a8004dc8a900803e2000d00888008b
:100cd0000368a9002368a80021e1a80021a1a900b8
:100ce00020c1a90020a1a8002081a8002021a900de
:100cf0004e08a8004e28a9004e48a8000388a90065
:100d0000a00e2000e00888002388a8002002a90087
:100d10002022a9002042a90020a2a9002062a90047
:100d20002082a90020e2a9002102a9002122a90015
:100d3000700720004011880022a2a90022c2a90049
:100d400022e2a90021e2a8002182a9004588a90089
:100d500045a8a80045c8a8002168a8002828a80020
:100d600023e2a9002342a8002362a9000188a90068
:100d70002188a8004608a9004628a8004648a800df
:100d80000e0ea80021e3a9002143a80021a3a90079
:100d90002123a9002103a90020e3a90020c3a90061
:100da00020a3a9002083a9002043a80023e3a900d1
:100db00023c3a90023a3a9002343a9002323a90037
:100dc0002303a90022c3a90022a3a9002283a9000a
:100dd0002263a9002243a9002223a9002203a9001b
:100de0002563ef0024e3ef003223ef002823ef0018
:100df0002623ef002e23ef003023ef0021a8a800c8
:100e000046c8a80046a8a9004688a80001a8a900cd
:100e100021e3a8004008a9004028a9004048a800f4
:100e20002008a8000008a900c208a80080c0b300dc
:100e3000c8e8b7002bc8a9002be8a9002c08a90016
:100e40000bc8a9000be8a9000c08a90001eca90037
:100e500001aca900016ca900014ca900012ca9005a
:100e6000010ca90000eca900008ca90000aca900ad
:100e700000cca900000ca900002ca900004ca9007e
:100e8000006ca900202cef00402cef00602cef003c
:100e90000000210020608800020ca900022ca9009b
:100ea000024ca900262cef00462cef00662cef0028
:100eb000282cef00482cef00682cef000aacef0064
:100ec00023eca80023cca80023aca900238ca90004
:100ed000236ca900234ca800232ca900230ca900f3
:100ee000222ca80043eca80043cca80043aca900e6
:100ef000438ca900436ca800434ca900432ca900d3
:100f0000430ca90063eca80063cca80063aca90063
:100f1000638ca800636ca800634ca900dabc2a00ab
:100f20001b32240030002c00fa608800fb6088002f
:100f300020618800dabc2a001b32240020402c00eb
:100f4000fa608800fb60880010618800dabc2a0023
:100f50001b32240030002c00fa608800fb608800ff
:100f600020628800dabc2a001b32240000802c009a
:100f7000fa608800fb60880010628800dabc2a00f2
:100f80001b32240030002c00fa608800fb608800cf
:100f900020638800dabc2a001b32240000802c0069
:100fa000fa608800fb60880010638800a7003700a3
:100fb0003f00370000202000006188000020200052
:100fc000006288000020200000638800020ca90055
:100fd000022ca800024ca80004acef0028acef00e3
:100fe00048acef0068acef00262cef00462cef0079
:100ff000662cef000aacef0023eca80023cca9007c
:1010000043eca80043cca90063eca80063cca90082
:10101000dabc2a001b32240030002c00fa60880061
:10102000fb60880020618800dabc2a001b322400a3
:1010300000002800fa608800fb60880010618800ca
:10104000dabc2a001b32240030002c00fa60880031
:10105000fb60880020628800dabc2a001b32240072
:1010600000002800fa608800fb6088001062880099
:10107000dabc2a001b32240030002c00fa60880001
:10108000fb60880020638800dabc2a001b32240041
:1010900000002800fa608800fb6088001063880068
:1010a00011eea90011aea900116ea900670037006a
:1010b000350037000010200000618800001020007b
:1010c000006288000010200000638800020ca90064
:1010d000022ca800024ca8000a2cef0004acef0080
:1010e000282cef005055250040628800a0aa2a0055
:1010f00040638800dabc2a001b32240030002c0038
:10110000fa608800fb60880020618800dabc2a0051
:101110001b32240000002c00fa608800fb6088006d
:1011200010618800dabc2a001b32240030002c0039
:10113000fa608800fb60880020628800dabc2a0020
:101140001b32240000002c00fa608800fb6088003d
:1011500010628800dabc2a001b32240030002c0008
:10116000fa608800fb60880020638800dabc2a00ef
:101170001b32240000002c00fa608800fb6088000d
:101180001063880031003700300037000010200065
:10119000006188000010200000628800020ca90095
:1011a000022ca800024ca8000a2cef0004acef00af
:1011b000282cef000000240040628800dabc2a00de
:1011c0001b32240030002c00fa608800fb6088008d
:1011d00020618800dabc2a001b32240000002c00a9
:1011e000fa608800fb60880010618800dabc2a0081
:1011f0001b32240030002c00fa608800fb6088005d
:1012000020628800dabc2a001b32240000002c0077
:10121000fa608800fb60880010628800dabc2a004f
:101220001b32240030002c00fa608800fb6088002c
:1012300020638800dabc2a001b32240000002c0046
:10124000fa608800fb60880010638800218ca90088
:10125000418ca900618ca900216ca900416ca900f6
:10126000616ca900214ca900414ca900614ca90066
:1012700020eca80040eca80060eca8003e2cef0099
:101280005e2cef007e2cef0001eca80080b2ef0096
:101290000000eb00a19d2100ff00090080587800ac
:1012a000a772ef00a872ef009632ef009832ef00bd
:1012b0000000eb00a1ad2100ff000900805878007c
:1012c000a972ef00aa72ef000080eb00619c210080
:1012d00009000900801878000000eb00612c210053
:1012e000ff00090080187800bb72ef00bc72ef00ad
:1012f0000000eb00614c2100ff000900801878001d
:10130000bd72ef000000eb00616c2100ff000900de
:1013100080187800be72ef00bf72ef00108ea90037
:10132000148ea900008ea900048ea90010aea90099
:1013300014aea9002008a8002068a80021a8a800d1
:1013400001a8a900f0ff2000306188002003a90057
:101350002023a80000122000e00888000388a900cc
:101360002388a800803e2000d00888000368a900d8
:101370002368a80000802000809388007e32ef0060
:101380007c32ef007a32ef0000c4b30082f2b70083
:1013900000c4b30084f2b700a0c0b30088f2b70065
:1013a0004000200050948800600020006094880075
:1013b000390707003808070097013700ff3ffc0096
:1013c0004200f8003600f8004400f8008e1f780054
:1013d0000e0020000d000900be1f78003200f8004a
:1013e0004012f8004212f8000100fc000008a900b9
:1013f0006612ae000c0037000021ef006612a90053
:101400006a32ef00be72ec00bed2bf000080fb006b
:101410000000d000616c21000100400001002000ac
:10142000010878001e003700000880004093880003
:101430005093800001002000f21f200003002000d4
:10144000000141008181490040938000010020009b
:10145000820f5000838f58000f0036000021ef00ec
:101460006a32ef00be72ec0042938000030020005d
:101470000000200011002000fafb0700e12b2100f2
:10148000914078008180fb0081804000626c2100e7
:10149000803079000200370040938000509388002c
:1014a000ff3ffc004212f9004012f9003200f9003f
:1014b000ae0120000d0009004f1778004f0778009b
:1014c0004400f9003600f9004200f9000100fc0078
:1014d00000400600ff3ffc004200f8003600f80024
:1014e0004400f8008e1f78000e0020000d00090057
:1014f000be1f78003200f8000100fc000068a9005f
:101500000021ef006612a800ff3ffc003200f90046
:10151000ae0120000d0009004f1778004f0778003a
:101520004400f9003600f9004200f9000100fc0017
:1015300000400600ff3ffc004200f8003600f800c3
:101540004400f8008e1f78000e0020000d000900f6
:10155000be1f78003200f8000100fc000108a9005d
:10156000ff3ffc003200f900ae0120000d00090031
:101570004f1778004f0778004400f9003600f90053
:101580004200f9000100fc0000400600ff3ffc00a3
:101590004200f8003600f8004400f8008e1f780082
:1015a0000e0020000d000900be1f78003200f80078
:1015b0004012f8000100fc000368a9001421ef00ac
:1015c0006c32ef005232ef00bed2bf00bf52e300d8
:1015d0000a003200bf72ec005232ec00bfd2bf00f2
:1015e0000080fb0000004000616c210060807800fa
:1015f0006c12b40060938800f3ff37005212e200cf
:101600000700360060938000929280000200e000a4
:1016100002003200110009000280d80060938800a7
:10162000800c200001002000b2948000c394800050
:101630000201400083814800b2ce8800c3ce8800fa
:10164000ba12a800ff3ffc004012f9003200f90076
:10165000ae0120000d0009004f1778004f077800f9
:101660004400f9003600f9004200f9000100fc00d6
:1016700000400600ff3ffc004200f8003600f80082
:101680004400f8008e1f78000e0020000d000900b5
:10169000be1f78003200f8000100fc000388a9009a
:1016a0001821ef002023a900ff3ffc003200f900c1
:1016b000ae0120000d0009004f1778004f07780099
:1016c0004400f9003600f9004200f9000100fc0076
:1016d00000400600ff3ffc004200f8003600f80022
:1016e0004400f8008e1f78000e0020000d00090055
:1016f000be1f78003200f8000100fc000168a9005c
:10170000a772ec00a7d2bf008080fb0030118000e0
:10171000a29d210080707900ff3ffc003200f9009b
:10172000ae0120000d0009004f1778004f07780028
:101730004400f9003600f9004200f9000100fc0005
:1017400000400600ff3ffc004200f8003600f800b1
:101750004400f8008e1f78000e0020000d000900e4
:10176000be1f78003200f8000100fc000828a90024
:101770002242ae00000037002222af002222a90040
:10178000ff3ffc003200f900ae0120000d0009000f
:101790004f1778004f0778004400f9003600f90031
:1017a0004200f9000100fc0000400600ff3ffc0081
:1017b0004200f8003600f8004400f8008e1f780060
:1017c0000e0020000d000900be1f78003200f80056
:1017d0000100fc000188a900128eaa00108ea90049
:1017e000ff3ffc003200f900ae0120000d000900af
:1017f0004f1778004f0778004400f9003600f900d1
:101800004200f9000100fc0000400600ff3ffc0020
:101810004200f8003600f8004400f8008e1f7800ff
:101820000e0020000d000900be1f78003200f800f5
:101830000100fc0001a8a9002003a90000188000f5
:10184000709388008093800071938000808f500097
:1018500004003600809380006e12b500c0938800ab
:1018600003003700709380007012b500c0938800a9
:10187000b09380007812b400a0938800c0938000d9
:10188000b0938800709380008093880080072000c8
:1018900001002000b2948000c39480000201400047
:1018a0008381480092ce8800a3ce8800ba12a80097
:1018b000ff3ffc003200f900ae0120000d000900de
:1018c0004f1778004f0778004400f9003600f90000
:1018d0004200f9000100fc0000400600ff3ffc0050
:1018e0004200f8003600f8004400f8008e1f78002f
:1018f0000e0020000d000900be1f78003200f80025
:101900000100fc000bc8a900ff3ffc003200f900f9
:10191000ae0120000d0009004f1778004f07780036
:101920004400f9003600f9004200f9000100fc0013
:1019300000400600ff3ffc004200f8003600f800bf
:101940004400f8008e1f78000e0020000d000900f2
:10195000be1f78003200f8000100fc000be8a9006f
:10196000ff3ffc003200f900ae0120000d0009002d
:101970004f1778004f0778004400f9003600f9004f
:101980004200f9000100fc0000400600ff3ffc009f
:101990004200f8003600f8004400f8008e1f78007e
:1019a0000e0020000d000900be1f78003200f80074
:1019b0000100fc000c08a900ff3ffc003200f90008
:1019c000ae0120000d0009004f1778004f07780086
:1019d0004400f9003600f9004200f9000100fc0063
:1019e00000400600a8d2bf00a752e3000700320063
:1019f000a872ec00a8d2bf000080fb00a19d2100ce
:101a000060c07800abf2b70001003700abf2ef0026
:101a1000000006000000060001948000e18f5000e5
:101a200000003a0050088000c09488003008800010
:101a3000b0948800ebff070080ceb300ab52b50036
:101a400006003900e0cfb300ab52b5000100390009
:101a500001003700ac72ef0094013700abf2ae002a
:101a600037003700ac72ef0070c8b300ab52e30030
:101a700005003a00abd2bf00acf2b700adf2ef0008
:101a8000aef2ef002d00370070c9b300ab52e30097
:101a900005003a00abd2bf00acf2b700aff2ef00e6
:101aa000b0f2ef002500370070cab300ab52e3007c
:101ab00005003a00abd2bf00acf2b700b1f2ef00c4
:101ac000b2f2ef001d00370070cbb300ab52e30061
:101ad00005003a00abd2bf00acf2b700b3f2ef00a2
:101ae000b4f2ef001500370070ccb300ab52e30046
:101af00004003a00abd2bf00acf2b700b5f2ef0081
:101b00000e00370070cdb300ab52e30004003a0082
:101b1000abd2bf00acf2b700b6f2ef00070037005f
:101b200070ceb300ab52e30004003a00abd2bf006a
:101b3000acf2b700b7f2ef00b8f2ef005b0137008c
:101b4000ac52e20002003a0058013700570137005a
:101b500070c8b300ac52e3003d003a0000e0ef0073
:101b6000ad52e30003003a00abd2bf00adf2b700c4
:101b700036003700abd2bf00aef2b700add2bf0027
:101b8000f1c2b30080cf100016003600e0c4b300ed
:101b9000ad52e30013003e00a972ec00a9d2bf00d1
:101ba0000080fb0072082000a1ad210002f0780047
:101bb000a972ec00a9d2bf000081fb00a1ad2100f9
:101bc000add2bf0000f17800a972ec00a9d2bf002d
:101bd0000081fb00a1ad2100aed2bf0000f1780072
:101be00019003700add2bf00f1c6b30080cf10009e
:101bf00015003600f0c7b300ad52e30012003e00fe
:101c0000a972ec00a9d2bf000080fb00720820007e
:101c1000a1ad210002f07800a972ec00a9d2bf00aa
:101c20000081fb00a1ad2100add2bf0000f1780022
:101c3000a972ec00a9d2bf000081fb00a1ad210078
:101c4000aed2bf0000f17800adf2ef00170137000f
:101c500070c9b300ac52e30073003a0000e0ef003b
:101c6000af52e30003003a00abd2bf00aff2b700bf
:101c70006c003700abd2bf00b0f2b700b052e20048
:101c800034003a00afd2bf00f1c2b30080cf1000e1
:101c900016003600e0c4b300af52e30013003e006c
:101ca000a972ec00a9d2bf000080fb0072092000dd
:101cb000a1ad210002f07800a972ec00a9d2bf000a
:101cc0000081fb00a1ad2100afd2bf0000f1780080
:101cd000a972ec00a9d2bf000080fb000200200026
:101ce000a1ad210002f0780019003700afd2bf008b
:101cf000f1c6b30080cf100015003600f0c7b30066
:101d0000af52e30012003e00a972ec00a9d2bf005e
:101d10000080fb0072092000a1ad210002f07800d4
:101d2000a972ec00a9d2bf000081fb00a1ad210087
:101d3000afd2bf0000f17800a972ec00a9d2bf00b9
:101d40000080fb0002002000a1ad210002f078001d
:101d500034003700afd2bf00f1c2b30080cf100013
:101d600016003600e0c4b300af52e30013003e009b
:101d7000a972ec00a9d2bf000080fb00720920000c
:101d8000a1ad210002f07800a972ec00a9d2bf0039
:101d90000081fb00a1ad2100afd2bf0000f17800af
:101da000a972ec00a9d2bf000081fb00a1ad210007
:101db000b0d2bf0000f1780019003700afd2bf00e9
:101dc000f1c6b30080cf100015003600f0c7b30095
:101dd000af52e30012003e00a972ec00a9d2bf008e
:101de0000080fb0072092000a1ad210002f0780004
:101df000a972ec00a9d2bf000081fb00a1ad2100b7
:101e0000afd2bf0000f17800a972ec00a9d2bf00e8
:101e10000081fb00a1ad2100b0d2bf0000f178002d
:101e2000aff2ef00a100370070cab300ac52e3007c
:101e300023003a0000e0ef00b152e30003003a0053
:101e4000abd2bf00b1f2b7001c003700abd2bf006d
:101e5000b2f2b700b1d2bf00f1c2b30080cf100020
:101e60001500360010c6b300b152e30012003e0068
:101e7000a972ec00a9d2bf000080fb00720a20000a
:101e8000a1ad210002f07800a972ec00a9d2bf0038
:101e90000081fb00a1ad2100b1d2bf0000f17800ac
:101ea000a972ec00a9d2bf000081fb00a1ad210006
:101eb000b2d2bf0000f17800b1f2ef007b00370032
:101ec00070cbb300ac52e3000a003a0000e0ef0030
:101ed000b352e30003003a00abd2bf00b3f2b70045
:101ee00003003700abd2bf00b4f2b700fa0207001c
:101ef0006e00370070ccb300ac52e30029003a000a
:101f000000e0ef00b552e30025003a00abd2bf007d
:101f1000b5f2b700b552e2000d003a00a972ec002c
:101f2000a9d2bf000080fb00720c2000a1ad2100ef
:101f300002f07800a972ec00a9d2bf000081fb007a
:101f4000a1ad2100b5d2bf0000f178001300370029
:101f5000b5d2bf00b1c0b30080cf10000f00360073
:101f600070c1b300b552e3000c003e00a972ec0052
:101f7000a9d2bf000080fb00720c2000a1ad21009f
:101f800002f07800a972ec00a9d2bf000081fb002a
:101f9000a1ad2100b5d2bf0000f17800b5f2ef008d
:101fa0004200370070cdb300ac52e30021003a008c
:101fb00000e0ef00b652e3001d003a00abd2bf00d4
:101fc000b6f2b700b652e20002003a00c472ef0067
:101fd0001600370010c0b300b652e3000a003a0002
:101fe00010d8250051002000b2948000c3948000d6
:101ff000020140008381480072ce880083ce8800b1
:10200000ba12a80009003700b6d2bf00f1c2b3006f
:1020100080cf10000500360010c6b300b652e300b2
:1020200002003e00b6d2bf00c4f2b700b6f2ef0025
:102030001e00370070ceb300ac52e3001b003a0024
:1020400000e0ef00b752e30003003a00abd2bf005c
:10205000b7f2b70015003700abd2bf00b8f2b70037
:10206000a972ec00a9d2bf000080fb00720e200014
:10207000a1ad210002f07800a972ec00a9d2bf0046
:102080000081fb00a1ad2100b7d2bf0000f17800b4
:10209000a972ec00a9d2bf000081fb00a1ad210014
:1020a000b8d2bf0000f17800b7f2ef007c12e20076
:1020b00058013a0098d2bf0092d2b6001040b20048
:1020c000930032009212a8009812ae009212a9005a
:1020d000bdd2bf000080fb0000004000614c210029
:1020e00060807800529480000200e000020032001c
:1020f000110009000280d80070948800719480005b
:10210000ee8f500002003600e0002000709488003e
:1021100072948000a0bd210060407900c0f2b70039
:10212000bbd2bf000080fb0000004000612c2100fa
:1021300060c07800c5f2b70088d2bf00c552e30086
:102140002d003600a972ec00a9d2bf000080fb0070
:1021500072092000a1ad210002f07800a972ec0004
:10216000a9d2bf000081fb00a1ad2100c0d2bf00f9
:1021700000f17800a972ec00a9d2bf000081fb0039
:10218000a1ad2100c5d2bf0000f17800c0d2bf00d0
:10219000c1f2b700d09380008c12bc00a2948800da
:1021a00020fe2f00a0948800a0948000fe0f500015
:1021b00002003400e0012000a0948800800220008a
:1021c0009412b400000678000c064600608c2100d2
:1021d00060007e00b2948000c39480000000410043
:1021e000e08049000001be0032ce880043ce880066
:1021f000ba12a80018003700c152e20016003600db
:10220000a972ec00a9d2bf000080fb007208200078
:10221000a1ad210002f07800a972ec00a9d2bf00a4
:102220000081fb00a1ad2100c1d2bf0000f1780008
:10223000a972ec00a9d2bf000080fb0002002000c0
:10224000a1ad210002f07800c172ef00c6b9ef0025
:10225000c8b9ef00ba12a8006612ae001600370027
:102260009052af0013003700a972ec00a9d2bf0052
:102270000080fb0072092000a1ad210002f078006f
:10228000a972ec00a9d2bf000080fb002207200049
:10229000a1ad210002f07800a972ec00a9d2bf0024
:1022a0000080fb00f2072000a1ad210002f07800c1
:1022b0009052a800150037009052ae00130037006e
:1022c000a972ec00a9d2bf000080fb0072082000b8
:1022d000a1ad210002f07800a972ec00a9d2bf00e4
:1022e0000080fb0022072000a1ad210002f0780051
:1022f000a972ec00a9d2bf000080fb000200200000
:10230000a1ad210002f078009052a900c100370071
:10231000010020009872af001140b0009232af006f
:102320001140b100560032009232a8009872ae00ff
:102330009232a900bdd2bf000080fb000000400027
:10234000614c2100608078006200200011000900cb
:102350000280d8007094880071948000f58f50003e
:1023600002003600500120007094880072948000b2
:10237000a0be210060407900c2f2b700bbd2bf000e
:102380000080fb0000004000612c210060c078004c
:10239000c5f2b70088d2bf00c552e3002100360065
:1023a000c452e2001d003a00c3d2bf00c252e30093
:1023b00019003200c572d500c572d500a972ec00b3
:1023c000a9d2bf000080fb00720a2000a1ad21004d
:1023d00002f07800a972ec00a9d2bf000081fb00d6
:1023e000a1ad2100c2d2bf0000f17800a972ec00bb
:1023f000c5d2bf000080fb00f005b000912a21008b
:10240000914078008180fb00a2ad210080707900ae
:10241000c2d2bf00c3f2b70001003700c372ef00a1
:1024200016003700c352e2001400360014aea900b3
:10243000a972ec00a9d2bf000080fb00720a200044
:10244000a1ad210002f07800a972ec00a9d2bf0072
:102450000081fb00a1ad2100c3d2bf0000f17800d4
:10246000a972ec00a9d2bf000080fb00020020008e
:10247000a1ad210002f07800c372ef0065003700c3
:102480000ac1bf0092d2b6004040b20061003200e3
:102490009252a8000a41ae009252a900bbd2bf00de
:1024a0000080fb0000004000612c210060c078002b
:1024b000c5f2b70088d2bf00c552e3002b0036003a
:1024c0009032ae0013003700a972ec00a9d2bf0011
:1024d0000080fb0072082000a1ad210002f078000e
:1024e000a972ec00a9d2bf000080fb009207200077
:1024f000a1ad210002f07800a972ec00a9d2bf00c2
:102500000080fb0002002000a1ad210002f0780055
:102510009032a9009012af0013003700a972ec00ae
:10252000a9d2bf000080fb0072092000a1ad2100ec
:1025300002f07800a972ec00a9d2bf000080fb0075
:1025400002072000a1ad210002f07800a972ec0082
:10255000a9d2bf000080fb00f2072000a1ad21003e
:1025600002f078009012a8002a0037009032af00e5
:1025700013003700a972ec00a9d2bf000080fb0055
:1025800072092000a1ad210002f07800a972ec00d0
:10259000a9d2bf000080fb0092072000a1ad21005e
:1025a00002f07800a972ec00a9d2bf000080fb0005
:1025b000f2072000a1ad210002f078009032a800bf
:1025c0009012ae0013003700a972ec00a9d2bf0030
:1025d0000080fb0072082000a1ad210002f078000d
:1025e000a972ec00a9d2bf000080fb000207200006
:1025f000a1ad210002f07800a972ec00a9d2bf00c1
:102600000080fb0002002000a1ad210002f0780054
:102610009012a900ba12af001101070050c0b30018
:10262000b952b500f9003100b2948000c394800023
:10263000d0948000e1948000800f5100818f590078
:10264000e90039009df2a800b952e20041003a00c9
:10265000c152e2003c003600d09380008c12bc00d6
:10266000a294880020fe2f00a0948800a0948000ef
:10267000fe0f500002003400e0012000a09488000a
:10268000800220009412b400000678000c06460078
:10269000608c210060007e00b2948000c3948000b2
:1026a00000004100e08049000001be0032ce8800f9
:1026b00043ce8800a972ec00a9d2bf000080fb00c5
:1026c00072092000a1ad210002f07800a972ec008f
:1026d000a9d2bf000081fb00a1ad2100c1d2bf0083
:1026e00000f17800a972ec00bbd2bf000080fb00b3
:1026f00000004000612c210060c07800912a210078
:10270000914078008180fb00a2ad210080707900ab
:10271000800220009412b400000678000c064600e7
:10272000608c210060007e00b2948000c394800021
:1027300000004100e08049000001be0032ce880068
:1027400043ce880002003700c6b9ef00c8b9ef00d9
:10275000a400370010c0b300b952e30018003a00db
:10276000c352e20013003600a972ec00a9d2bf00e8
:102770000080fb00720a2000a1ad210002f0780069
:10278000a972ec00a9d2bf000081fb00a1ad21001d
:10279000c3d2bf0000f17800a972ec00a9d2bf003b
:1027a0000080fb0002002000a1ad210002f07800b3
:1027b000c372ef00cab9ef00ccb9ef00890037004f
:1027c00020c0b300b952e30005003a00c40107007d
:1027d0008032ef00ceb9ef00d0b9ef0081003700b2
:1027e00030c0b300b952e3003a003a0012958000bd
:1027f0002395800020852b00e1f72300c2f7070016
:102800002092880031928800a093800037f807005a
:102810000001be00a0702d0031ba2300baf70700f6
:10282000229280003392800059f7070010958800ab
:1028300021958800bb72ec001295800023958000e2
:102840000000200001082400aff7070017f7070079
:1028500007f80700801f7800bbd2bf000081fb0093
:1028600002014100612c21004fb17800bbd2bf00b2
:102870000080fb0000004000612c21006080780097
:1028800000928800bbd2bf008080fb0084d2bf00d2
:102890000080fb00008650000c064600602c2100e2
:1028a00060007e004012b50030948800bbd2bf00ab
:1028b0000080fb0000004000612c21006080780057
:1028c0004400dd0030638800d2b9ef00d4b9ef00d6
:1028d0004400370040c0b300b952e30041003a0061
:1028e000bbd2bf000080fb0000004000612c210033
:1028f000608078008000780088d2bf000080fb00f4
:10290000810f5000030036006c12e2000100360017
:102910006c32ed00f2948000039580003033230088
:1029200031f7230078f70700209288003192880061
:1029300060938000edf707000001be00d0cc2c00b2
:10294000c1d4230070f707002292800033928000e8
:102950000ff70700f094880001958800bd72ec0025
:10296000f094800001958000c1f70700801f780077
:10297000bdd2bf000081fb0002014100614c21007b
:102980004fb17800bdd2bf008080fb0082d2bf0073
:102990000080fb00008650000c064600604c2100c1
:1029a00060007e00d1f707000001be00f0948000b7
:1029b00001958000f5f6070088f70700d09388009e
:1029c000bdd2bf000080fb0000004000614c210030
:1029d000608078004500dd0030628800d6b9ef00e5
:1029e000d8b9ef001e00070099f2ae0006003700cc
:1029f0000621ef000a21ef000080eb00619c21001e
:102a000009000900801878000400370099f2ae0030
:102a1000020037000621ef000a21ef00a9d2bf0013
:102a2000aa52e300090032000188af000700370016
:102a3000aa72ec00aad2bf000080fb00a1ad210069
:102a400060c078000080fb00201188009832af0041
:102a500014cea8009832ae0014cea900f1fb3700c6
:102a6000b9f2ef009df2a8005032ef008192800091
:102a7000e48f500016003e0080928000c200dd000e
:102a8000609c2100008040001000be000001be00dc
:102a9000d0948000e1948000800f5100818f590014
:102aa0000900310080928000c200dd00609c21009e
:102ab000008040001000be00d0948800e19488009f
:102ac00050d2bf00b9f2b7005032ec00e7ff390036
:102ad000ba12a90000000600b3f2bf0016003200cf
:102ae00070c0b300b352e30013003e00a972ec00c3
:102af000a9d2bf000080fb00720b2000a1ad210015
:102b000002f07800a972ec00a9d2bf000081fb009e
:102b1000a1ad2100b3d2bf0000f17800a972ec0092
:102b2000a9d2bf000081fb00a1ad2100b4d2bf003b
:102b300000f17800e8003700b0c0b300b352e30002
:102b400013003a00a972ec00a9d2bf000080fb007c
:102b5000720b2000a1ad210002f07800a972ec00f8
:102b6000a9d2bf000080fb00b2002000a1ad21006f
:102b700002f07800a972ec00a9d2bf000081fb002e
:102b8000a1ad2100b4d2bf0000f17800d20037001f
:102b9000b3d2bf00d1c0b30080cf10001600360002
:102ba00030c1b300b352e30013003e00a972ec0041
:102bb000a9d2bf000080fb00720b2000a1ad210054
:102bc00002f07800a972ec00a9d2bf000081fb00de
:102bd000a1ad2100b3d2bf0000f17800a972ec00d2
:102be000a9d2bf000081fb00a1ad2100b4d2bf007b
:102bf00000f17800b800370000c4b300b352e3001e
:102c000013003a00a972ec00a9d2bf000080fb00bb
:102c1000720b2000a1ad210002f07800a972ec0037
:102c2000a9d2bf000080fb0002042000a1ad21005a
:102c300002f07800a972ec00a9d2bf000081fb006d
:102c4000a1ad2100b4d2bf0000f17800a20037008e
:102c500010c4b300b352e30019003a00b452e200ca
:102c6000140036007cb2ef00a972ec00a9d2bf00bc
:102c70000080fb00720b2000a1ad210002f0780063
:102c8000a972ec00a9d2bf000080fb00b2072000af
:102c9000a1ad210002f07800a972ec00a9d2bf001a
:102ca0000080fb0002002000a1ad210002f07800ae
:102cb000010037007c32ef007e32ef0086003700e3
:102cc00020c4b300b352e30025003a00a972ec001f
:102cd000a9d2bf000080fb00720b2000a1ad210033
:102ce00002f07800a972ec00a9d2bf000080fb00be
:102cf00022042000a1ad210002f07800a972ec00ae
:102d0000a9d2bf000081fb00a1ad2100b4d2bf0059
:102d100000f17800b452e20010003a005032ef00a7
:102d200081928000e48f500009003e008092800074
:102d3000c200dd00609c210000814000f0ff2f00f8
:102d4000f1ff2f000089be005032ec00f4ff390083
:102d5000ba12a8007e32ef007cb2ef005e003700ae
:102d600060c4b300b352e3000a003a00b4d2bf001b
:102d70000080fb0000004000209288004452ec00dc
:102d800082f2b700209280001040b00082f2b700bb
:102d90005100370070c4b300b352e3000a003a0098
:102da000b4d2bf000080fb000000400020928800e9
:102db0004452ec0084f2b700209280001040b00032
:102dc00084f2b7004400370090c4b300b352e3006c
:102dd0000b003a00f0c7b300b452b5000500310053
:102de000b4d2bf000080fb004500dd0030618800e8
:102df00002003700f0ff2000306188003600370005
:102e0000a0c4b300b352e30003003a00b4d2bf0041
:102e100088f2b70030003700d0c4b300b352e300eb
:102e200010003a00b4d2bf0080407800f0072000c4
:102e300001405000b4f2b700f2002000b4d2bf004d
:102e40000080fb000200e0000200320011000900d7
:102e50000280d800209288004412ec005094880030
:102e60001d003700e0c4b300b352e30005003a0090
:102e7000b4d2bf000080fb000020ec00609488000a
:102e800015003700b0c7b300b352e30012003a0098
:102e9000a972ec00a9d2bf000080fb00720b2000d9
:102ea000a1ad210002f07800a972ec00a9d2bf0008
:102eb0000080fb00b2072000a1ad210002f07800e5
:102ec000a972ec00a9d2bf000080fb000200200024
:102ed000a1ad210002f07800b3f2ef00000006007f
:102ee000a972ec00a9d2bf000080fb00720b200089
:102ef000a1ad210002f07800a972ec00a9d2bf00b8
:102f00000080fb0012002000a1ad210002f078003b
:102f1000a972ec00a9d2bf000080fb004201200092
:102f2000a1ad210002f07800a972ec00a9d2bf0087
:102f30000080fb00720b2000a1ad210002f07800a0
:102f4000a972ec00a9d2bf000080fb002200200083
:102f5000a1ad210002f07800a972ec00a9d2bf0057
:102f60000080fb0082072000a1ad210002f0780064
:102f7000a972ec00a9d2bf000080fb00720b2000f8
:102f8000a1ad210002f07800a972ec00a9d2bf0027
:102f90000080fb0032002000a1ad210002f078008b
:102fa000a972ec00a9d2bf000080fb001200200033
:102fb000a1ad210002f07800a972ec00a9d2bf00f7
:102fc0000080fb00720b2000a1ad210002f0780010
:102fd000a972ec00a9d2bf000080fb0052002000c3
:102fe000a1ad210002f07800a972ec00a9d2bf00c7
:102ff0000080fb0012002000a1ad210002f078004b
:10300000a972ec00a9d2bf000080fb00720b200067
:10301000a1ad210002f07800a972ec00a9d2bf0096
:103020000080fb0062002000a1ad210002f07800ca
:10303000a972ec00a9d2bf000080fb0012002000a2
:10304000a1ad210002f07800a972ec00a9d2bf0066
:103050000080fb00720b2000a1ad210002f078007f
:10306000a972ec00a9d2bf000080fb007200200012
:10307000a1ad210002f07800a972ec00a9d2bf0036
:103080000080fb00f2072000a1ad210002f07800d3
:103090007eb2ef0000000600c6b8ef00a0c7250012
:1030a00040c688005098250050c688004081250001
:1030b00060c68800906a250070c6880030542500dc
:1030c00080c68800303e250090c6880090282500e4
:1030d000a0c6880050132500b0c6880060fe2400fa
:1030e000c0c68800c0e92400d0c6880080d524006e
:1030f000e0c6880090c12400f0c68800f0ad24002e
:1031000000c78800a09a240010c78800a087240068
:1031100020c78800f074240030c788009062240023
:1031200040c788008050240050c78800b03e24006b
:1031300060c78800302d240070c78800f01b240071
:1031400080c78800000b240090c7880050fa230035
:10315000a0c78800e0e92300b0c78800c0d92300d9
:10316000c0c78800e0c92300d0c7880040ba230048
:10317000e0c78800e0aa2300f0c78800c09b2300b6
:1031800000c88800e08c230010c88800307e23002f
:1031900020c88800d06f230030c88800a0612300b9
:1031a00040c88800b053230050c88800f045230071
:1031b00060c888007038230070c88800202b230066
:1031c00080c88800101e230090c88800401123008a
:1031d000a0c8880090042300b0c8880020f822000e
:1031e000c0c88800e0eb2200d0c88800d0df2200f1
:1031f000e0c88800f0d32200f0c8880050c8220040
:1032000000c98800d0bc220010c9880080b122000b
:1032100020c9880070a6220030c98800809b220047
:1032200040c98800c090220050c988002086220032
:1032300060c98800c07b220070c9880080712200ac
:1032400080c988006067220090c98800805d2200e4
:10325000a0c98800c0532200b0c98800204a2200bb
:10326000c0c98800b0402200d0c988006037220061
:10327000e0c98800402e2200f0c9880040252200c5
:1032800000ca8800601c220010ca8800b013220007
:1032900020ca8800200b220030ca8800b002220019
:1032a00040ca880060fa210050ca880040f221001c
:1032b00060ca880030ea210070ca880050e221000c
:1032c00080ca880090da210090ca8800e0d22100ec
:1032d000a0ca880060cb2100b0ca8800f0c32100da
:1032e000c0ca8800b0bc2100d0ca880080b52100c7
:1032f000e0ca880080ae2100f0ca880090a72100b3
:1033000000cb8800b0a0210010cb8800009a2100db
:1033100020cb88006093210030cb8800e08c210016
:1033200040cb88008086210050cb8800308021006f
:1033300060cb8800007a210070cb8800f0732100f8
:1033400080cb8800f06d210090cb880000682100c0
:10335000a0cb880040622100b0cb8800805c2100b7
:10336000c0cb8800e0562100d0cb880060512100fe
:10337000e0cb8800f04b2100f0cb88009046210084
:1033800000cc88005041210010cc8800203c210056
:1033900020cc88001037210030cc8800103221006a
:1033a00040cc8800202d210050cc880040282100ee
:1033b00060cc88008023210070cc8800d01e2100c2
:1033c00080cc8800301a210090cc8800a015210004
:1033d000a0cc880020112100b0cc8800c00c2100b6
:1033e000c0cc880070082100d0cc880020042100c7
:1033f000e0cc8800f0ff2000f0cc8800d0fb20005b
:1034000000cd8800c0f7200010cd8800d0f3200048
:1034100020cd8800e0ef200030cd880000ec2000b7
:1034200040cd880030e8200050cd880070e42000b6
:1034300060cd8800c0e0200070cd880020dd200035
:1034400080cd880090d9200090cd880010d6200033
:10345000a0cd8800a0d22000b0cd880040cf2000b1
:10346000c0cd8800e0cb2000d0cd8800a0c82000cf
:10347000e0cd880060c52000f0cd880030c220007b
:1034800000ce880010bf200010ce880000bc2000b5
:1034900020ce88000000060010c3b300dafbb7009e
:1034a00030c3b300dbfbb70050c3b300dcfbb70095
:1034b00070c3b300ddfbb70090c3b300defbb70001
:1034c000b0c3b300dffbb700d0c3b300e0fbb7006d
:1034d000f0c3b300e1fbb70010c4b300e2fbb700d8
:1034e00030c4b300e3fbb70050c4b300e4fbb70043
:1034f00070c4b300e5fbb70090c4b300e6fbb700af
:10350000b0c4b300e7fbb700d0c4b300e8fbb7001a
:1035100070c3b300eafbb70090c3b300ebfbb70086
:10352000b0c3b300ecfbb700d0c3b300edfbb700f2
:10353000f0c3b300eefbb70010c4b300effbb7005d
:1035400030c4b300f0fbb70050c4b300f1fbb700c8
:1035500070c4b300f2fbb70090c4b300f3fbb70034
:10356000b0c4b300f4fbb700d0c4b300f5fbb700a0
:10357000f0c4b300f6fbb70010c5b300f7fbb7000b
:1035800030c5b300f8fbb70050c5b300f9fbb70076
:1035900070c5b300fafbb70090c5b300fbfbb700e2
:1035a000b0c5b300fcfbb700d0c5b300fdfbb7004e
:1035b000f0c5b300fefbb70010c6b300fffbb700b9
:0835c00000000600ffff3700c8
:020000040000fa
:1035c80040120000100000008000000050120000af
:1035d8004600000080000000961200001000000065
:1035e80080000000a61200002000000080000000fb
:1035f800c61200000007000080000000c619000085
:103608001400000080000000da1900002602000003
:0836180080000000000000002a
:00000001FF
